:1000000010C01FC01EC01DC01CC03FC01AC093C07E
:1000100025C017C016C015C014C013C012C011C02F
:1000200010C011241FBECFE5D1E0DEBFCDBF20E060
:10003000A0E6B0E001C01D92A738B207E1F7AAD050
:100040009BC1DECF1DBC1CBC8FB5836C8FBD89E00E
:100050008EBD85E28CB984E08BB908951F920F9212
:100060000FB60F9211248F939F93809180009091EF
:100070008100019690938100809380009F918F91E1
:100080000F900FBE0F901F9018951F920F920FB6F2
:100090000F9211242F938F939F93AF93BF938091CF
:1000A000600090916100A0916200B09163000196A0
:1000B000A11DB11D8093600090936100A093620028
:1000C000B093630020918600213059F5809373002E
:1000D00090937400A0937500B093760084B595B5A5
:1000E00090937D0080937C008091800090918100AE
:1000F00090937F0080937E00589B10C080917C007D
:1001000090917D008115924048F480917E009091FD
:100110007F00019690937F0080937E0082E0809321
:100120008600BF91AF919F918F912F910F900FBE3D
:100130000F901F9018951F920F920FB60F921124D7
:100140008F939F9388B599B588519C4F99BD88BD71
:10015000809164008F5F8C3018F4809364000BC032
:1001600010926400809171009091720001969093BA
:100170007200809371009F918F910F900FBE0F902E
:100180001F901895809590959370F8949BBD8ABDAB
:100190007894089580E886BD16BC80E48ABBDF9A17
:1001A00010928600109277004DDF7894C1E062983B
:1001B0008091710090917200883E934028F01092D7
:1001C000770080E090E0DEDF629A6298809186009E
:1001D00081110CC080917100909172000A9730F0EB
:1001E000C09386001092720010927100629A809102
:1001F00086008230E1F680917E0090917F00209110
:100200007C0030917D00A0E0B0E04AE0880F991FAB
:10021000AA1FBB1F4A95D1F7820F931FA11DB11DC5
:100220008093780090937900A0937A00B0937B003C
:100230008091780090917900A0917A00B0917B0034
:100240004091650050916600609167007091680070
:10025000841B950BA60BB70B8093820090938300B1
:10026000A0938400B09385008091780090917900EC
:10027000A0917A00B0917B00809365009093660016
:10028000A0936700B0936800809173009091740010
:10029000A0917500B09176004091690050916A007C
:1002A00060916B0070916C00841B950BA60BB70BD3
:1002B00080936D0090936E00A0936F00B0937000D8
:1002C0008091730090917400A0917500B0917600B8
:1002D0008093690090936A00A0936B00B0936C00C8
:1002E0001092860080917700882309F442C06091C3
:1002F0006D0070916E0080916F0090917000809001
:10030000820090908300A0908400B09085002FD14F
:1003100020E03BE147E35BE4BCD16B017C01C5011C
:10032000B40125D19B01AC01C701B6018CD0F62EDA
:10033000072F182FD92F2DEC38E14CE955E4A5D122
:1003400018162CF48DECF82E08E11CE9D5E426E40F
:1003500037EB41E55EE36F2D702F812F9D2F99D1F3
:1003600020E030E040E05FE30AD0D5D0CB010ADFE7
:100370001ECFC09377001BCFF8941AC25058BB27EA
:10038000AA270ED048C139D130F03ED120F031F447
:100390009F3F11F41EF42EC10EF4E095E7FB24C13B
:1003A000E92F4AD180F3BA176207730784079507CC
:1003B00018F071F49EF562C10EF4E0950B2EBA2F81
:1003C000A02D0B01B90190010C01CA01A00111245B
:1003D000FF27591B99F0593F50F4503E68F11A1607
:1003E000F040A22F232F342F4427585FF3CF469598
:1003F00037952795A795F0405395C9F77EF41F16BA
:10040000BA0B620B730B840BBAF09150A1F0FF0F83
:10041000BB1F661F771F881FC2F70EC0BA0F621F6F
:10042000731F841F48F4879577956795B795F7955F
:100430009E3F08F0B3CF9395880F08F09927EE0FF1
:100440009795879508950CD0E6C0DED040F0D5D0C2
:1004500030F021F45F3F19F0C7C0511110C1CAC07C
:10046000EBD098F39923C9F35523B1F3951B550BA2
:10047000BB27AA2762177307840738F09F5F5F4F77
:10048000220F331F441FAA1FA9F333D00E2E3AF0B8
:10049000E0E830D091505040E695001CCAF729D0D2
:1004A000FE2F27D0660F771F881FBB1F2617370721
:1004B0004807AB07B0E809F0BB0B802DBF01FF2751
:1004C00093585F4F2AF09E3F510568F08DC0D7C00A
:1004D0005F3FECF3983EDCF3869577956795B7958B
:1004E000F7959F5FC9F7880F911D9695879597F9A6
:1004F0000895E1E0660F771F881FBB1F621773071F
:100500008407BA0720F0621B730B840BBA0BEE1F33
:1005100088F7E095089598D088F09F5790F0B92F0C
:100520009927B751A0F0D1F0660F771F881F991F48
:100530001AF0BA95C9F712C0B13081F09FD0B1E07E
:1005400008959CC0672F782F8827B85F39F0B93F8E
:10055000CCF3869577956795B395D9F73EF490954A
:100560008095709561957F4F8F4F9F4F0895E894C8
:1005700009C097FB3EF490958095709561957F4FEB
:100580008F4F9F4F9923A9F0F92F96E9BB27939599
:10059000F695879577956795B795F111F8CFFAF4A9
:1005A000BB0F11F460FF1BC06F5F7F4F8F4F9F4FDA
:1005B00016C0882311F096E911C0772321F09EE838
:1005C000872F762F05C0662371F096E8862F70E09E
:1005D00060E02AF09A95660F771F881FDAF7880F78
:1005E0009695879597F9089597F99F6780E870E049
:1005F00060E008959FEF80EC089500240A94161699
:10060000170618060906089500240A941216130600
:10061000140605060895092E0394000C11F488238E
:1006200052F0BB0F40F4BF2B11F460FF04C06F5FAA
:100630007F4F8F4F9F4F089557FD9058440F551F80
:1006400059F05F3F71F04795880F97FB991F61F054
:100650009F3F79F087950895121613061406551FCB
:10066000F2CF4695F1DF08C0161617061806991F37
:10067000F1CF86957105610508940895E894BB272C
:1006800066277727CB0197F908956ED008F48FEF8E
:1006900008950AD0C0CFB1DF28F0B6DF18F0952357
:1006A00009F0A2CFA7CFEBCFC7DFA8F39923D9F3E7
:1006B0005523C9F3950F50E0551FAA27EE27FF27B2
:1006C000BB2700240894679520F4E20FF31FB41FA2
:1006D0000A1E220F331F441FAA1F6695A9F777959C
:1006E00030F4F30FB41F0A1E121E08F46395330F83
:1006F000441FAA1F221F769599F7879520F4B40FFF
:100700000A1E121E631F440FAA1F221F331F869545
:10071000A9F7862F712D602D11249F5750408AF024
:10072000E1F088234AF0EE0FFF1FBB1F661F771F03
:10073000881F91505040A9F79E3F510570F054CF4B
:100740009ECF5F3FECF3983EDCF3869577956795F7
:10075000B795F795E7959F5FC1F7FE2B880F911D21
:100760009695879597F90895990F0008550FAA0B4C
:10077000E0E8FEEF16161706E807F907C0F01216B4
:100780001306E407F50798F0621B730B840B950BB7
:1007900039F40A2661F0232B242B252B21F408950C
:1007A0000A2609F4A140A6958FEF811D811D0895A9
:0407B000F894FFCFEB
:00000001FF
